:020000040802F0
:10000000B06F0020A10102084D2E0208ED26020863
:10001000392E0208AD080208D53D02080000000094
:100020000000000000000000000000005D37020832
:100030008D1D020800000000B12F0208B53802082B
:10004000BB010208BB010208BB010208BB01020898
:10005000BB010208BB010208BB010208BB01020888
:100060002D1E02085D1E0208711E0208BB01020857
:10007000BB010208BB010208BB010208BB01020868
:10008000BB010208BB010208BB010208BB01020858
:10009000BB010208BB010208BB010208A11E020845
:1000A000BB010208BB010208BB010208BB01020838
:1000B000BB01020821390208BB010208BB0102088A
:1000C000BB010208BB010208BB010208BB01020818
:1000D000BB010208BB010208BB010208BB01020808
:1000E000911D0208BB010208BB010208BB01020806
:1000F000BB010208BB010208BB010208BB010208E8
:10010000BB010208BB010208BB010208BB010208D7
:10011000BB010208BB010208BB010208BB010208C7
:10012000BB010208BB010208BB010208BB010208B7
:10013000BB010208BB010208BB010208BB010208A7
:10014000BB010208BB010208BB010208BB01020897
:10015000BB010208BB010208BB010208653A0208A4
:10016000BB010208BB010208BB010208BB01020877
:10017000BB010208BB010208BB010208BB01020867
:10018000BB010208BB010208DFF810D000F046F8FE
:1001900000480047593F0208AFF30080B06F0020CD
:1001A0000648804706480047FEE7FEE7FEE7FEE711
:1001B000FEE7FEE7FEE7FEE7FEE7FEE7B9380208E6
:1001C0008901020840EA01039B0703D009E008C93E
:1001D000121F08C0042AFAD203E011F8013B00F80C
:1001E000013B521EF9D27047D2B201E000F8012B58
:1001F000491EFBD270470022F6E710B513460A46A7
:1002000004461946FFF7F0FF204610BD421C10F8C7
:10021000011B0029FBD1801A70470000064C074DD6
:1002200006E0E06840F0010394E8070098471034C6
:10023000AC42F6D3FFF7ACFF144102083441020888
:1002400070B58C1810F8015B15F0070301D110F898
:10025000013B2A1106D110F8012B03E010F8016BC5
:1002600001F8016B5B1EF9D12B0705D40023521E48
:100270000DD401F8013BFAE710F8013BCB1A921CB0
:1002800003E013F8015B01F8015B521EF9D5A142AE
:10029000D8D3002070BD70B506460C46154608E060
:1002A0003046721C96B200F007F804F8010B681E85
:1002B00085B2002DF4D170BD2DE9F0410446002532
:1002C000002702F087FCA02002F050FC02F0D4FCD2
:1002D000054605B129E0201202F048FC02F0CCFCF2
:1002E000054605B121E02646E11704EB116109122C
:1002F000A4EB0121C8B202F039FC02F0BDFC0546B6
:1003000005B112E002F066FCA12002F02FFC02F021
:10031000B3FC054605B108E0002002F0F1FB0746FA
:1003200002F07EFC3846BDE8F08102F079FC002046
:10033000F9E72DE9F04105460C46164600270CE08A
:100340002178284600F010F80746012F02D000203F
:10035000BDE8F081681C85B2641C301EA6F1010165
:100360008EB2EDD10120F3E72DE9F04104460E46AF
:10037000002702F02FFCA02002F0F8FB02F07CFC2A
:100380000746201202F0F2FB02F076FC07462546F3
:10039000E11704EB11610912A4EB0121C8B202F0CC
:1003A000E5FB02F069FC0746304602F0DFFB02F095
:1003B00063FC074602F034FC0F2003F03BFD0120F4
:1003C000BDE8F0811CB502F045FB01211F2003F0C0
:1003D0007FF80620009001208DF8040000208DF8A1
:1003E000060003208DF8050001208DF807006946FE
:1003F0002A4801F0DAFF4FF460400090694628482F
:1004000001F0D3FF4FF4E05000906946254801F019
:10041000CCFF43F6010000906946234801F0C5FF78
:1004200041F2100000906946204801F0BEFF04210F
:100430001A4802F030F84FF40051194802F02BF836
:100440000121194802F027F84FF48051164802F0B4
:1004500022F84FF48051154802F01DF802210F4890
:1004600002F019F81021114802F015F80220104985
:100470000860012100F01CFA0421002000F018FAA5
:1004800047F6FF7001F00CFE47F6FF7001F01EFE0C
:1004900000F0C0F802F0D0F91CBD000000000240DE
:1004A0000004024000080240000C0240001002401C
:1004B0008C0000201CB50121102003F009F8042055
:1004C000009001208DF8040000208DF80600032024
:1004D0008DF8050001208DF807006946034801F0FA
:1004E00064FF012002F098F91CBD000000100240DA
:1004F00010B5002440480078012819D13F48006811
:1005000020F0FF003D4908603D48407809680843F5
:100510003A49086001213B48007800F0C9F90421FC
:100520003648006800F0C4F90020334908700124FF
:100530003548007801281AD13048006820F47F40FF
:100540002E4908602E484078096841EA00202B496E
:10055000086001212B48007800F0AAF904212748FF
:10056000006800F0A5F900202749087001242748F9
:10057000007801281AD12148006820F47F001F4923
:1005800008601F484078096841EA00401B4908603C
:1005900001211C48007800F08BF9042117480068FD
:1005A00000F086F9002019490870012418480078E5
:1005B00001281AD11148006820F07F400F490860D7
:1005C0000F484078096841EA00600C490860012141
:1005D0000C48007800F06CF904210848006800F02D
:1005E00067F900200A4908700124012C02D1642017
:1005F00003F040FC10BD0000900000209800002097
:1006000003010020940000209100002092000020AF
:100610009300002000B585B00820009000208DF8E0
:10062000040003208DF8050002208DF807006946BC
:10063000334801F0BAFE4FF400600090694631483B
:1006400001F0B3FE4FF48070009069462E4801F02F
:10065000ACFE2020009069462C4801F0A6FE012146
:10066000880302F045FF0B21022003F079F80821EE
:10067000032003F075F80321002003F071F8052131
:10068000042003F06DF840F62810029000208DF849
:100690000C0008208DF80D0001208DF80E0002A836
:1006A00001F0B4FC09208DF8100001208DF8110034
:1006B00000208DF8120001208DF8130004A802F02C
:1006C000C7FB17208DF8100001208DF811008DF860
:1006D00012008DF8130004A802F0BAFB28208DF850
:1006E000100001208DF8110003208DF81200012068
:1006F0008DF8130004A802F0ABFB05B000BD0000AC
:100700000000024000080240000C024000100240BD
:100710002DE9FF5F05460C462F78EE782879697938
:1007200000EB01201FFA80F8A879E97900EB01209D
:100730001FFA80F98DF808608DF80B40ADF809803C
:1007400001208DF80C0001AADDE9020101F082FF11
:1007500083469DF80410584600F06CFF8DF8086041
:100760008DF80B40ADF8099000208DF80C00012C9D
:1007700000D100BF022C00D100BF6A46DDE90201B2
:1007800001F068FF82469DF80000032802DB9DF817
:10079000000000909DF80010504600F04BFF2246EC
:1007A0003946022001F01CFABDE8FF9F01461329DB
:1007B00001DA00207047A1F109000A2290FBF2F350
:1007C00002FB130008B10020F4E70120F2E700006B
:1007D0002DE9FE4F04460D46277894F8018094F8E1
:1007E000029094F803A0207A617A00EB01201FFAAE
:1007F00080FB002000908DF80880ADF804B08DF8E3
:1008000009908DF807708DF806A0012D00D100BF6A
:100810006A46DDE9010101F041FE06460EB9BDE878
:10082000FE8F681EC100009888400549096808438A
:1008300003490860042D00D100BF00BFEFE70000AE
:10084000880000202DE9F04105462F781548006802
:1008500000F00040134908600026002410E047FA29
:1008600004F000F0010050B1621CD1B206EB860327
:100870006A1C02EB4300FFF7ABFF701CC6B2641C9E
:10088000042CECDB01210848006800F011F8042179
:100890000448006800F00CF8022003F0CBFABDE831
:1008A000F0810000880000208C00002000BFFEE7DF
:1008B0002DE9F04104460E4600250027012E2BD1DC
:1008C00000BF26E004F0800747B14FF48051324862
:1008D00001F0E1FD012003F0CDFA07E04FF4805173
:1008E0002D4801F0D6FD012003F0C4FA4FF48041F9
:1008F0002A4801F0D0FD012003F0BCFA4FF48041FA
:10090000264801F0C6FD012003F0B4FA6400681C1B
:10091000C5B2082DD6DB3CE0042E3AD1002526E0F6
:1009200004F0004747B14FF480511B4801F0B3FD7C
:10093000012003F09FFA07E04FF48051164801F0C0
:10094000A8FD012003F096FA4FF48041134801F00E
:10095000A2FD012003F08EFA4FF480410F4801F010
:1009600098FD012003F086FA6400681CC5B2202DB2
:10097000D6DB4FF40041094801F08DFD012003F062
:1009800079FA4FF40041054801F083FD012003F09E
:1009900071FABDE8F0810000000802400004024046
:1009A0002DE9F04106460F4690461C46012577206A
:1009B0000449087022462946012003F025F9BDE8C4
:1009C000F0810000B44600202DE9F05F81468A46A0
:1009D00093461E46812739463448FFF70CFC01F048
:1009E00081FE044620783149087060784870A0780C
:1009F0008870002005E0211D0A5CC11C2B4B5A5455
:100A0000401C0E28F7DB04F11200FFF7FFFB054640
:100A1000102D01DD102000E028460546002007E0EB
:100A200004F112010A5C00F11101204B5A54401CE0
:100A3000A842F5DB04F12200FFF7E8FB0546202D74
:100A400001DD202000E028460546002007E004F1F3
:100A500022010A5C00F12101144B5A54401CA842A7
:100A6000F5DB04F14200FFF7D1FB0546402D01DD27
:100A7000402000E028460546002007E004F142013E
:100A80000A5C00F14101094B5A54401CA842F5DBB5
:100A9000074B3A460549032000F0FCFC80463246ED
:100AA0003946022003F0B0F8BDE8F09FB4460020BC
:100AB000B44E00202DE9F04FA9B081468A469346F6
:100AC0001E46812739463648FFF795FB684603F0F6
:100AD0001DFA6C4620783249087060784870A0781A
:100AE0008870002005E0211D0A5CC11C2C4B5A5463
:100AF000401C0E28F7DB04F11200FFF787FB0546C8
:100B0000102D01DD102000E028460546002007E0FA
:100B100004F112010A5C00F11101214B5A54401CEE
:100B2000A842F5DB04F12200FFF770FB0546202DFB
:100B300001DD202000E028460546002007E004F102
:100B400022010A5C00F12101154B5A54401CA842B5
:100B5000F5DB04F14200FFF759FB0546402D01DDAE
:100B6000402000E028460546002007E004F142014D
:100B70000A5C00F141010A4B5A54401CA842F5DBC3
:100B8000084B3A460649032000F084FC8046324672
:100B90003946032003F038F829B0BDE8F08F000093
:100BA000B4460020B44E00202DE9F041AAB006461C
:100BB0000F4690461C460E2501A803F0A7F92A46C9
:100BC0000DF18E010548FFF7FDFA22462946042063
:100BD00003F01AF82AB0BDE8F0810000B446002006
:100BE00003F0A8F9012080F3138800BF00BFBFF312
:100BF0004F8F0748006800F4E06006490843001D75
:100C000003490860BFF34F8F00BF00BFFEE700003D
:100C10000CED00E00000FA052DE9F04105460C4618
:100C20001646984627465EB12146284601F09AFDB1
:100C300008B9BDE8F081204604EBD071C1F34F073D
:100C4000142F07DA002003E0295C034A1154401CEA
:100C5000B842F9DB00BFECE7200100202DE9F041AC
:100C600006460F4690461C4614252A460549064866
:100C7000FFF7A8FA22462946072002F0C5FFBDE883
:100C8000F081000020010020B44600202DE9F0434F
:100C9000A9B005460C4616469946012704F0FF0800
:100CA00056B1204604EBD071C1F3470821462846CF
:100CB00001F058FD00B90027B8F10E0F00DA002747
:100CC00067B1684603F022F90E2229460DF18A0029
:100CD000FFF778FA684603F023F903E001210220C8
:100CE00000F08CFC29B0BDE8F0832DE9F04104460A
:100CF0000D4616461F460121902000F07FFCBDE8FE
:100D0000F08170472DE9FF4F85B004460E464248FA
:100D1000007810B109B0BDE8F08F01203E4908709D
:100D2000324621463D48FFF74DFA3046FFF73EFD7B
:100D300038B90020384908700121052000F05EFC18
:100D4000E8E7A6F10800C5B2281D00F0FF08615DC4
:100D5000681C205C01EB0021A81C205C01EB004119
:100D6000E81C205C01EB0060049014F8081008F106
:100D70000100205C01EB00201FFA80FB2946204681
:100D800001F0DAFC03902946204601F038FD814647
:100D9000DDE90310884201D1CB4507D000201E4970
:100DA00008700121FF2000F029FCB3E74FF0000A92
:100DB000207802902046FFF745FD002712E00298B8
:100DC000384100F0010060B17A1CD1B20AEB8A030D
:100DD000621C02EB4300FFF79BFC0AF1010000F0EC
:100DE000FF0A7F1C042FEADB02200190002006E0AE
:100DF000B11E0144615C0A4A1154411CC8B2022868
:100E0000F6DB2220089A019902F0FEFE002002493A
:100E1000087000BF7EE70000840000207C5F002097
:100E2000B44600202DE9F0470546884691469A468B
:100E30004A464146284601F0AFF928B9012105206C
:100E400000F0DCFBBDE8F0872F78002600240FE0DF
:100E500047FA04F000F0010048B1621CD1B206EB81
:100E6000C6036A1C981801F047F9701CC6B2641CCE
:100E7000042CEDDB00BFE5E72DE9F0470546884689
:100E800091469A462E780027002420E046FA04F086
:100E900000F00100D0B1012000EB8400285C00F0DC
:100EA0000101022000EB8400285C61F35F1007461B
:100EB00032463946042000F093FE042000EB840003
:100EC0002F5C32463946052000F08AFE641C042C53
:100ED000DCDB00F0A1FBBDE8F08700002DE9F04766
:100EE0008046894692461D4608261348008884B2EB
:100EF000200A124908704C701148008884B2200AF8
:100F00008870CC700F48008884B2200A08714C7138
:100F10000D48008884B2200A8871CC710B4B324690
:100F2000302000F0B7FA07462A463146302002F05A
:100F30006BFEBDE8F0870000BC000020B446002036
:100F4000BE000020C0000020C2000020B44E0020DF
:100F50002DE9F04105460E4617461C462146012064
:100F600002F004FDBDE8F0812DE9F04104460D4694
:100F700016461F460121902000F040FBBDE8F0819D
:100F80002DE9F05F07460C4615461E464FF0010856
:100F900004F0FF095DB1204604EBD071C1F34709AD
:100FA0002146384601F0DEFB08B94FF00008B9F1E0
:100FB000010F01D04FF00008B8F1000F05D1012159
:100FC000052000F01BFBBDE8F09F4FF0640A0749C5
:100FD000384601F0EEFF824601F0BFFF83463246FD
:100FE0005146332002F010FE00BFECE7B44600206B
:100FF0002DE9F04104460E461546984601272B463A
:101000003A463146204601F0D0FB28B901210220A2
:1010100000F0F4FABDE8F081207802F027FA00BF72
:10102000F8E700002DE9F05F06460C4617469B46A0
:101030004FF0010804F0FF095FB1204604EBD071C6
:10104000C1F347092146304601F08CFB08B94FF047
:101050000008B9F1050F01DA4FF00008B8F1000FF0
:1010600017D096F800A001200D49087000250DE06A
:101070004AFA05F000F0010038B1681CC1B2701CDA
:1010800000F0E0F90A2002F0F5FE6D1C042DEFDB04
:1010900003E00121052000F0B1FABDE8F09F000057
:1010A000840000202DE9F05F06460C4617469B465B
:1010B0004FF0010904F0FF0A5FB1204604EBD07144
:1010C000C1F3470A2146304601F04CFB08B94FF006
:1010D0000009BAF1050F01DA4FF00009B9F1000F6C
:1010E0001ED0012004E0315C01EB0828411CC8B28D
:1010F0000528F8DB3078801FC5B225B901214046AC
:1011000000F086FB05E0012D03D10221404600F0EE
:101110007FFB022D03D10321404600F079FB03E061
:101120000121052000F06AFABDE8F09F2DE9F05F8B
:1011300006460D4617469B464FF0010905F0FF0A8B
:101140005FB1284605EBD071C1F3470A2946304606
:1011500001F008FB08B94FF00009BAF1020F01DAFB
:101160004FF00009B9F1000F05D10121052000F071
:1011700045FABDE8F09F96F801803478012C05D13E
:1011800001224146022000F02BFD16E0022C05D181
:1011900002224146104600F023FD0EE0042C05D14A
:1011A00003224146022000F01BFD06E0082C04D17A
:1011B00004224146022000F013FD142002F05AFEE2
:1011C00000BFD6E72DE9F047044688461746994602
:1011D0003B4606224146204601F0E7FA28B90121A4
:1011E000052000F00BFABDE8F0876078217800EB6D
:1011F00001260025022004E0215C01EB0525411CAD
:10120000C8B20628F8DB07490E70074805600121BF
:101210003046FFF74DFB04212846FFF749FB00BF8E
:10122000E1E7000094000020980000202DE9F04143
:1012300005460E4614461F462346122231462846CE
:1012400001F0B3FA28B90121052000F0D7F9BDE873
:10125000F0811221284601F071FD00BFF7E7000080
:101260002DE9F0479AB006460C4617469A464FF0CD
:10127000010804F0FF094FB1204604EBD071C1F31F
:1012800047092146304601F06DFA8046B9F1070F53
:1012900001DA4FF00008B8F1000F06D10121052056
:1012A00000F0ACF91AB0BDE8F0871648007800B13C
:1012B000F8E7012013490870652C0ADA002004E0E1
:1012C000FF2122180DF80210401CC4F16501814273
:1012D000F6DC224631466846FEF774FF0DF1010147
:1012E000684601F0BBFE0546012D02D100F094F9DD
:1012F00003E00121FF2000F081F90020014908707E
:1013000000BFCFE7840000202DE9F04104460D46E0
:1013100016461F4602F078FBBDE8F081F8B504469A
:101320000D4616461F4600F077F902F077FE0020C2
:101330000090F8BD00F070F900BFFEE72DE9F0471E
:1013400005460C46174698464FF0010904F0FF0A7F
:101350005FB1204604EBD071C1F3470A214628460D
:1013600001F000FA08B94FF00009BAF1020F01DAF2
:101370004FF00009B9F1000F05D10121052000F05F
:101380003DF9BDE8F0870226287820B1012804D075
:10139000022806D103E0292604E0082602E00826F8
:1013A00000E000BF00BF06F10801FF221448FEF76D
:1013B0001BFF287820B1012808D0022816D10DE0A3
:1013C000312210490E48FEF7FDFE10E00C480E4990
:1013D000096801600D490968416008E008480C4946
:1013E000096801600B490968416000E000BF00BF67
:1013F00042463146E32002F007FC00BFC1E700008F
:10140000B44600207C5F0020180100201C01002051
:10141000A8020020A40200202DE9F04104460F4656
:1014200090461D468026802221460548FEF7CAFECA
:101430002A463146E42002F0E7FBBDE8F0810000D7
:10144000B44600202DE9FE4304460D462678677811
:10145000A078E17800EB01201FFA80F80EB9012690
:1014600000E000268DF800708DF80350ADF8018083
:101470008DF8046002AADDE9000101F0EBF8814675
:101480009DF80810484600F0D5F8012002F0D2FC83
:10149000BDE8FE832DE9F04106460F4615461C4681
:1014A00055202070AA206070BB20A070E6702571C6
:1014B000280A6071002D04DD2A463946A01DFEF77A
:1014C00081FE0D21A81D21540A21E81D2154401C34
:1014D000BDE8F0812DE9F0413A483B49097830F800
:1014E00011604FF6FF70864200D15FE04FF6FF704B
:1014F0003449354A127821F8120000200CE03349B3
:10150000895D334A1154711C44F2080291FBF2F3D5
:1015100002FB13118EB2401CB0F5026FEFDB2C48BA
:101520000078552807D12A484078AA2803D12848AE
:101530008078BB2800D039E0254DA888801D294639
:10154000085C0D2804D1A888C01D085C0A2800D0BA
:101550002CE01C481C49097830F811601C4F00240D
:1015600020E004EB44001B4911F82000F978884280
:1015700016D104EB4400DFF85C8008EB8000437A6E
:1015800004EB440008EB8000027AB98804EB4400C5
:1015900008EB8000D0F804C00D48801DE04703E050
:1015A000601CC4B21E2CDCDB00BF00BF0648007804
:1015B000401C142190FBF1F201FB1200024908705B
:1015C000BDE8F08134570020AD000020AC060020BB
:1015D0005C5700203401002070B5142401252246F8
:1015E00004490548FEF7EEFD2A462146072002F091
:1015F0000BFB70BD20010020B446002070B50446EE
:101600000D460126034804702A463146B02002F0F8
:10161000FBFA70BDB446002010B50224C020044976
:10162000087048700122214602F0EEFA10BD000059
:10163000B44600202DE9F04704460E460027B84680
:101640000025A946012E04D0022E19D0032E48D120
:1016500030E001216B4800F01CFF012002F00AFC81
:101660000121684800F017FF012002F003FC01216E
:10167000644800F00EFF012002F0FCFB012531E080
:101680004FF40051604800F004FF012002F0F2FB2B
:101690004FF400515C4800F0FEFE012002F0EAFB2E
:1016A0004FF40051584800F0F4FE012002F0E2FB34
:1016B000022517E00421554800F0EBFE012002F05E
:1016C000D9FB0421514800F0E6FE012002F0D2FBD4
:1016D00004214E4800F0DDFE012002F0CBFB032583
:1016E00000E000BF00BF4FF4C051474800F0D3FEF8
:1016F000012002F0BFFB4FF40061434800F0C9FE37
:10170000012002F0B7FB4FF480513F4800F0C1FECA
:10171000012002F0AFFB00274AE04FF000082AE06A
:1017200004F00049B9F1000F08D04FF400613648C9
:1017300000F0B1FE012002F09DFB07E04FF40061D4
:10174000314800F0A6FE012002F094FB4FF48051D6
:101750002D4800F0A0FE012002F08CFB4FF48051D8
:10176000294800F096FE022002F084FB640008F194
:10177000010000F0FF08B8F1080FD1DB4FF4006161
:10178000214800F086FE012002F074FB4FF48051E6
:101790001D4800F080FE012002F06CFB4FF48051E8
:1017A000194800F076FE022002F064FB781CC7B2F4
:1017B000042FB2DB4FF48051134800F06CFE01207F
:1017C00002F058FB4FF400610F4800F064FE012066
:1017D00002F050FB012D03D101210A4800F05BFE0D
:1017E000022D03D12903084800F055FE032D03D133
:1017F0000421064800F04FFE012002F03BFB0025CB
:10180000BDE8F087000C02400004024000000240E6
:101810002DE9F04704460D460027C4F3034848F07D
:101820003009A6B2012D04D0022D04D0032D06D11B
:1018300003E0182705E01A2703E01C2701E0BDE8B4
:10184000F08700BF01F062F8384601F02BF801F094
:10185000A9F800B149E0484601F024F801F0A2F8E7
:1018600000B142E0300A01F01DF801F09BF800B130
:101870003BE0F0B201F016F801F094F800B134E06A
:1018800001F06AF8012D04D0022D0ED0032D26D1CF
:1018900019E00121174800F0FCFD052002F0EAFAEA
:1018A0000121144800F0F7FD1AE04FF400511248EE
:1018B00000F0EFFD052002F0DDFA4FF400510E4874
:1018C00000F0E9FD0CE004210C4800F0E2FD0520E9
:1018D00002F0D0FA0421094800F0DDFD00E0AEE797
:1018E00000BF012002F0A6FAA9E701F035F800BF19
:1018F000A5E70000000C0240000402400000024086
:1019000010B500241448006820F440101249086003
:1019100008460068086004E0601CC4B2012002F0C0
:10192000A9FA0E48006808B1C82CF5DBC82C01DB09
:10193000012010BD002404E0601CC4B2012002F0AC
:1019400099FA0648006808B9F02CF5DBF02C01DBA9
:101950000120EEE70020ECE70008024028024142A7
:1019600010B5002400F0B0F800F08CF8FFF7C8FFC5
:10197000CC2000F0B5F8BE2000F0B2F800F03CF842
:1019800004B2200104B22046E11704EB11710C11DE
:1019900001480480204610BDBC0000201CB540F268
:1019A0000140009001208DF8040000208DF8060011
:1019B00002208DF8050001208DF8070069460B48CC
:1019C00000F0F3FC4FF4007000906946084800F006
:1019D000ECFC4FF4007000906946064800F0E5FC0E
:1019E00000F050F8FFF78CFF1CBD0000000802401B
:1019F000000C02400010024070B50026002408E0F0
:101A000000F00CF8054605FA04F0304386B2601C7D
:101A1000C4B20C2CF4DB304670BD000010B50024BD
:101A20001548006820F44010134908600846006813
:101A300040F480100860002010490860022002F085
:101A400019FA01200E49C1F8A8020B48006820F4D9
:101A50004010094908600846006808600C2002F040
:101A600009FA06488038006800B10124322002F0EB
:101A700001FA204610BD000000080240A8024142C1
:101A80000000414210B50D48006820F440100B4999
:101A900008600846006840F480100860002008498B
:101AA000086040F2EE2002F0E5F901200549C1F896
:101AB000A8020F2002F0DEF910BD0000000802406D
:101AC000A80241420000414210B5FFF7DBFFFFF7DB
:101AD00017FFCC2000F004F8442000F001F810BDFE
:101AE00070B504463648006820F440103449086058
:101AF0000846006840F4801008603248006820F40E
:101B00004020304908600846006840F480200860A2
:101B10002D48006820F440202B49086008460068E2
:101B200040F4802008602648006820F00300244923
:101B300008600846006840F00100086001253CE0AC
:101B400004F001066410DEB100202049086020493D
:101B5000C1F8A4021F4908601F49C1F88002022091
:101B600002F088F90120194908601C4908601949E8
:101B700008601949C1F880023C2002F07BF91AE0A4
:101B80000020124908601249C1F8A40211490860F6
:101B90001149C1F880023C2002F06CF901200B4988
:101BA00008600E4908600B4908600B49C1F88002C3
:101BB000022002F05FF9681CC5B2082DC0DD70BDBF
:101BC00000080240000C024000100240A8024142FE
:101BD00000804142A402424200004142A4824142AC
:101BE0002DE9F04707460E46904600250024B946E9
:101BF000B8F1010F09D0B8F1020F0DD0B8F1030F01
:101C000011D0B8F1040F1AD113E04FF480515C48A1
:101C100000F041FC012413E04FF48051594800F0DA
:101C20003AFC03240CE00221574800F034FC052460
:101C300006E01021534800F02EFC062400E000BF0F
:101C400000BF022002F016F9012C04D121034C48F8
:101C500000F01FFC14E0032C05D14FF480514948DB
:101C600000F017FC0CE0052C04D10221464800F0DE
:101C700010FC05E0062C03D11021424800F009FCBD
:101C8000022002F0F7F800252BE009F0800ABAF1F3
:101C9000800F08D14FF40061394800F0FCFB0220AE
:101CA00002F0E8F807E04FF40061354800F0F1FB7E
:101CB000022002F0DFF84FF40051314800F0EBFB56
:101CC000022002F0D7F84FF400512D4800F0E1FB5C
:101CD000022002F0CFF84FEA49604FEA1069681C11
:101CE000C5B2082DD1DB002529E006F0800ABAF143
:101CF000800F08D14FF40061214800F0CCFB022096
:101D000002F0B8F807E04FF400611D4800F0C1FB95
:101D1000022002F0AFF84FF40051194800F0BBFB6D
:101D2000022002F0A7F84FF40051154800F0B1FB73
:101D3000022002F09FF87006060E681CC5B2082D3E
:101D4000D3DB012C03D121030D4800F0A4FB032CAD
:101D500004D14FF480510B4800F09DFB052C03D1BA
:101D60000221094800F097FB062C03D110210548F9
:101D700000F091FB022002F07DF8BDE8F087000042
:101D8000000C0240001002400000024070470000BA
:101D900010B54FF4806000F02DF9012814D1142003
:101DA00002F048F84FF400411B4800F069FB30B9DD
:101DB0001A480078012802D10020184908704FF411
:101DC000806000F011F925E04FF4805000F012F926
:101DD000012814D1142002F02DF84FF4805110483E
:101DE00000F04EFB30B90F480078012802D10020E6
:101DF0000C4908704FF4805000F0F6F80AE04FF4F8
:101E0000006000F0F7F8012804D107490870C0020B
:101E100000F0EAF810BD0000000C0240A90000200C
:101E200000000240A80000209000002010B51420FF
:101E300002F000F80421074800F022FB30B9064800
:101E40000078012802D1002003490870042000F026
:101E5000CBF810BD000C0240A700002010B50120F7
:101E600002490870082000F0BFF810BD9200002061
:101E700010B5142001F0DEFF1021074800F000FB30
:101E800030B906480078012802D1002003490870C3
:101E9000102000F0A9F810BD000C0240A6000020A0
:101EA00010B5402000F0A6F8012812D1142001F04E
:101EB000C1FF4021124800F0E3FA30B91148007820
:101EC000012802D100200F490870402000F08CF852
:101ED00015E0202000F08EF8012805D10A4908708D
:101EE000202000F081F80AE04FF4807000F082F8C2
:101EF000012804D105490870000200F075F810BDF2
:101F0000000C0240A500002093000020910000205A
:101F10000EB50121880301F0EBFA0221032001F044
:101F20001FFC0421032001F01BFC0621032001F00B
:101F300017FC0821032001F013FC0A21002001F006
:101F40000FFC0C21002001F00BFC0521042001F006
:101F500007FC41F27450009000208DF80400082026
:101F60008DF8050001208DF80600684600F04EF857
:101F700008208DF8080001208DF8090002208DF856
:101F80000A0001208DF80B0002A800F061FF0A2072
:101F90008DF8080002208DF8090001208DF80A0054
:101FA0008DF80B0002A800F053FF28208DF80800E0
:101FB00003208DF8090002208DF80A0001208DF819
:101FC0000B0002A800F044FF17208DF80800042041
:101FD0008DF8090002208DF80A0001208DF80B0011
:101FE00002A800F035FF0EBD0149086070470000EF
:101FF000143C014001460020034A12680A400AB11D
:10200000012000E000207047143C014000212349DA
:102010008279002A3AD00A46126803689A430B462E
:102020001A600A1D126803689A430B1D1A60027930
:1020300011440A6803681A430A60184A0832126891
:1020400003689A43154B08331A601A1D1268036817
:102050009A43124B0C331A604279102A0ED11A1F80
:10206000126803681A430D4B08331A601A1D126870
:1020700003681A43094B0C331A600DE00749427993
:1020800011440A6803681A430A6005E002791144A2
:102090000A6803689A430A6070470000003C0140E8
:1020A0002DE9F041054602260C274FF00108064CA9
:1020B00044EA076444EA08442C4331462046FFF7CB
:1020C000B9FABDE8F0810000000030102DE9F041C0
:1020D000054602260C274FF00308064C44EA076425
:1020E00044EA08442C4331462046FFF7A3FABDE8F2
:1020F000F0810000000030102DE9FF5F0446657894
:10210000A678E77894F808802079617900EB0120BF
:102110001FFA80F9A079E17900EB01201FFA80FA1B
:1021200000201B4908601B480068019000200090B7
:102130008DF80C508DF80D608DF80A708DF80E80BA
:102140006B4601AADDE9020100F03CFA8346BBF1CF
:10215000000F01D1BDE8FF9F9DF800000C49086009
:102160000C4901980860012109480068FEF7A0FBAE
:10217000042108480068FEF79BFB4846FFF7A6FFCE
:102180005046FFF78DFF022001F054FE00BFE1E74B
:102190008C000020880000202DE9F04106460D4605
:1021A00017460A2D02DA0020BDE8F0810024002045
:1021B00009E00121814032781140012901D1611CDF
:1021C000CCB2411CC8B20428F3DB681E04EBC40186
:1021D000884201D00020E7E74FB104EBC400401C67
:1021E00000F0FF084146304600F0BCFADCE7012071
:1021F000DAE7000001490860704700000C3C02402B
:1022000030B10749096841F48061054A116005E071
:102210000349096821F48061014A11607047000098
:10222000003C024070B504460A460026092502B962
:1022300009E0012A01D1160205E0022A01D11602A5
:1022400001E04FF4407600F09FF80546092D28D1B3
:102250001548006820F4407013490860084600687B
:10226000304308600846006820F0F800086008461F
:10227000006844F0020108430B4908600846006802
:1022800040F48030086000F07FF80546064800689A
:1022900020F00200044908600846006820F0F800B9
:1022A0000860284670BD0000103C02400920134918
:1022B000096801F48031B1F5803F01D101201CE0B3
:1022C0000E49096801F0100109B1062015E00B491B
:1022D000096801F4807109B102200EE0074909681C
:1022E00001F0EF0109B1072007E00449096801F096
:1022F000020109B1082000E0092070470C3C0240AF
:102300000348006840F00040014908607047000041
:10231000103C024030B502460C46092500F034F866
:102320000546092D19D10E48006820F440700C496B
:1023300008600846006840F40070086008460068BD
:1023400040F001000860146000F01EF805460448E3
:10235000006820F0010002490860284630BD0000F6
:10236000103C02400548006800F0004028B10448D5
:1023700002490C390860034808607047103C02406D
:1023800023016745AB89EFCD08B509200090FFF721
:102390008DFF009002E0FFF789FF00909DF800009C
:1023A0000128F8D09DF8000008BDF0B50A460021CC
:1023B0000023002400BF3DE0012505FA01F3156864
:1023C00005EA03049C4234D105684F000326BE4051
:1023D000B543056015794E00B54006683543056084
:1023E0001579012D02D01579022D16D185684F007F
:1023F0000326BE40B543856055794E00B5408668DA
:1024000035438560456801268E40B5434560456883
:1024100096798E40B6B235434560C5684F000326B5
:10242000BE40B543C560D5794E00B540C66835435A
:10243000C560491C1029BFD3F0BDF0B500230024AE
:102440004D07ED0E02FA05F3CE1000F1200555F808
:1024500026504E07F70E0F26BE40B543CF1000F1B1
:10246000200646F82750CE1000F1200555F82650DA
:1024700045EA0304CE1000F1200545F82640F0BDE2
:102480000246002013690B400BB1012000E0002040
:1024900070474183704701837047000017B50021E2
:1024A0000023BDF800004FF6FF74A04203D143485B
:1024B000007801431BE0BDF80000B0F57A7F03D13E
:1024C0003E484078014312E0BDF80000B0F5FA7FC5
:1024D00003D13A488078014309E0BDF80000142890
:1024E00003D13648C078014301E000201EBD9DF8AD
:1024F000050038B99DF80200012803D13048007862
:10250000014318E09DF8050038B99DF8020020B994
:102510002B484078014301230DE09DF80500012878
:1025200007D19DF8020020B9254880780143012396
:1025300001E00020DAE7F3B19DF80400012802D0A1
:102540009DF8040000B935E09DF80400142802D17C
:1025500041F008012EE09DF80400052802D141F069
:10256000400127E09DF80400642802D141F04801B1
:1025700020E00020BAE79DF80400012802D09DF871
:10258000040000B916E09DF80400052802D141F0CE
:1025900008010FE09DF80400142802D141F0480121
:1025A00008E09DF80400642802D141F0480101E0F0
:1025B00000209BE71160012098E700000301002044
:1025C000000100200FB502219DF8060000F0010077
:1025D00008B141F080019DF8050000B91BE09DF8AD
:1025E0000500012802D141F0080114E09DF8050022
:1025F000022804D1106840F0004010600BE09DF804
:102600000500032804D1106880F00040106002E04B
:10261000002004B000BD9DF80200012802D141F065
:10262000400105E09DF8020000B901E00020F0E75C
:102630009DF80400012800D108E09DF80400052859
:1026400002D141F0200101E00020E2E719700120F1
:10265000DFE70000F7B5042503269DF80470012F7D
:1026600001D1022501261D489DF800700FB92F46A3
:1026700000E0374639469DF803707F1EC7EB071709
:10268000DFF85CC0674401EB410C17F80C707F1F4A
:1026900017709DF803707F1EC7EB0717DFF840C067
:1026A000674401EB410C6744BB789DF803707F1EC3
:1026B000C7EB0717DFF828C0674401EB410C6744FC
:1026C0007C7840EA036040EA0440BDF8017038437A
:1026D0001778012F00D100BFFEBD000000003010B0
:1026E000C400002000487047000000200248034951
:1026F000086000BFFEE700000400FA050CED00E0F2
:10270000002111E00846082208E000F001031BB197
:10271000074B83EA500000E04008521E002AF4DC18
:10272000044B43F82100491CFF29EBDD70470000F2
:102730002083B8EDAC02002030B502460B464FF0C6
:10274000FF31002008E0CCB2155C6C40044D55F818
:10275000244084EA1121401C9842F4D3C84330BD80
:10276000AC02002030B5034609B9012030BD08464F
:1027700001EBD0725210A1EB42020AB10020F5E742
:10278000084601EBD072C2F34F04002209E0985CC6
:10279000C043C0B215195D5DA84201D00020E5E735
:1027A000521CA242F3DB0120E0E72DE9F043814611
:1027B0000C4615461E4614B90120BDE8F0830127DA
:1027C00004F0FF0856B1204604EBD071C1F347086E
:1027D00021464846FFF7C6FF00B90027A84500D0AC
:1027E00000273846E9E710B50246002004E0135CF4
:1027F000DB4344181355401C8842F8DB10BD10B56C
:1028000002460023002003E0145C1C44A3B2401CD9
:102810008842F9D3184610BD10B50446012C04D1E6
:1028200004210448FFF737FE03E004210148FFF7C5
:1028300030FE10BD001002401CB50121022000F046
:1028400047FE4FF4C050009001208DF80400002096
:102850008DF8060003208DF8050001208DF8070093
:1028600069460B48FFF7A1FD01200A4908600A49A3
:10287000C1F8AC0201210948FFF70DFE4FF40051E9
:102880000348FFF708FE04210548FFF704FE1CBDBE
:1028900000040240B082404200804042000C0240EE
:1028A0000000024070B504461548006820F440005E
:1028B000134908600846006840F480000860002062
:1028C00010490860002517E0E0090E49091F08605B
:1028D0006006040E022001F0CDFA01200A49C1F879
:1028E000B002022001F0C6FA00200649086002206A
:1028F00001F0C0FA681CC5B2082DE5DB70BD000010
:1029000000040240B08240420080404210B50F48AF
:10291000006820F440000D4908600846006840F453
:102920008000086001200A4908600A49C1F8B00225
:10293000042001F09FFA002005490860042001F0FE
:1029400099FA00200349C1F8B00210BD000402400A
:10295000AC8240420080404210B50F48006820F42D
:1029600040000D4908600846006840F48000086097
:1029700000200A4908600A49C1F8AC02042001F0AD
:1029800079FA0120054908600549C1F8AC02042024
:1029900001F070FA10BD000000040240B082404215
:1029A0000080404210B500241348006820F4400025
:1029B0001149086008460068086001200F49086056
:1029C00001F058FA01200E49C1F8B00201F052FAA4
:1029D00007E0601CC4B2FA2C03DDFFF7BDFF012045
:1029E00010BD0648803800680028F2D10349091D4F
:1029F000086000BFF4E7000000040240AC824042DF
:102A00000080404210B500200F4908600F48006860
:102A100020F440400D4908600846006840F48040BA
:102A2000086000200A49C1F89C020A2001F022FA3D
:102A30000120054908600A2001F01CFA0020044921
:102A4000C1F8980210BD0000988240420004024084
:102A5000008040421CB50121022000F039FDE02039
:102A6000009001208DF8040000208DF8060003205E
:102A70008DF8050000208DF8070069460948FFF72A
:102A800094FC0020084908600A2001F0F3F90120B5
:102A90000649C1F894020449091D08600349C1F8B8
:102AA0009C021CBD000402409482404200804042CF
:102AB00010B500200F4908600F48006820F440401E
:102AC0000D4908600846006840F480400860012015
:102AD0000A49C1F89C020A2001F0CCF901200549FD
:102AE00008600A2001F0C6F900200449C1F89802E4
:102AF00010BD000098824042000402400080404225
:102B000070B5054600241648006820F4404014497A
:102B10000860084600680860002616E00020114999
:102B200008600A2001F0A6F901200F49C1F89802B7
:102B30006006040E0B487C38006808B1601CC4B203
:102B40000A2001F097F9701CC6B2082EE6DB15B911
:102B5000FFF7AEFF01E0FFF755FF204670BD000014
:102B600000040240988240420080404270B5044612
:102B70001548006820F44040134908600846006882
:102B800040F480400860002010490860002517E0EC
:102B9000E0090E49091D08606006040E0A2001F0D4
:102BA00069F901200A49C1F898020A2001F062F986
:102BB0000020064908600A2001F05CF9681CC5B2D3
:102BC000082DE5DB70BD0000000402409882404201
:102BD0000080404210B50F48006820F440400D4985
:102BE00008600846006840F48040086001200A49F7
:102BF00008600A49C1F898020A2001F03BF9002058
:102C0000054908600A2001F035F900200349C1F8A0
:102C1000980210BD000402409C8240420080404265
:102C200010B5022001F026F91048006820F4404059
:102C30000E4908600846006840F4804008600020A3
:102C40000B4908600B49C1F89C020A2001F012F9F7
:102C5000012007490860052001F00CF90120054911
:102C6000C1F89C020A2001F005F910BD00040240E1
:102C7000988240420080404210B50024114800680C
:102C800020F440400F4908600846006808600A20A8
:102C900001F0F0F801200C4908600A2001F0EAF880
:102CA00007E0601CC4B2FA2C03DDFFF7B9FF012076
:102CB00010BD05487C3800680028F2D10249086040
:102CC00000BFF5E700040240988240424CF6CC4039
:102CD00001490860704700000030004010B500F066
:102CE00013F810BD70B505460C4645F2555000F07E
:102CF0001FF8284600F010F8204600F013F800F006
:102D000003F8FFF7E3FF70BD4AF6AA200149086007
:102D100070470000003000400149486070470000E3
:102D200000300040014988607047000000300040DA
:102D300001490860704700000030004070B505464A
:102D40000E46002410E02A5D02F0010104F1260283
:102D5000D0B200F017F82A5D52105100621CD0B2B8
:102D600000F010F8601CC4B2B442ECDB00F001F8D3
:102D700070BD10B50121252000F004F8142001F0E9
:102D800079F810BD70B506460D460024102000F0FD
:102D9000F8F8C82001F06EF8FFF71CFF7820FFF765
:102DA000E5FEFFF769FF044604B110E03046FFF787
:102DB000DDFEFFF761FF044604B108E02846FFF797
:102DC000D5FEFFF759FF044604B100E000BFFFF74E
:102DD00027FFC82001F04EF870BD000010B5134861
:102DE000134908604FF4A06000F06EF80121022042
:102DF00000F06EFBA82000F0FFFFFA210420FFF78F
:102E000071FF4FF4E13001F029F9FDF753FBFEF7B4
:102E1000C5FD00F077F9FDF7D5FAFFF779F8002046
:102E200000F024FB01200349087010BD00000208D7
:102E300008ED00E0AA00002002480349086000BF36
:102E4000FEE700000400FA050CED00E0704700000A
:102E500070B5002100230F22C4781CB3174C2468DE
:102E600004F4E064C4F5E064C4F30721C1F1040490
:102E7000E3B20A4144789C40E1B284781440214393
:102E80000C07210E0E4C05786155047804F01F05DF
:102E90000124AC4005786D11AD0005F1E025C5F8C1
:102EA000004109E0047804F01F050124AC40054D01
:102EB0000678761145F8264070BD00000CED00E064
:102EC00000E400E080E100E002490143024A1160B1
:102ED000704700000000FA050CED00E070B5822498
:102EE0000325FFF777FE2046FFF740FEFFF7C4FEFD
:102EF00000B10EE02846FFF739FEFFF7BDFE00B136
:102F000007E00020FFF732FEFFF7B6FE00B100E059
:102F100000BFFFF785FE70BD70B50446822501260F
:102F2000FFF758FE2846FFF721FEFFF7A5FE00B188
:102F300010E03046FFF71AFEFFF79EFE00B109E0F1
:102F400004F00101881CFFF711FEFFF795FE00B1A8
:102F500000E000BFFFF764FE70BD70B50024FFF70E
:102F600039FEE1252846FFF701FEFFF785FE002028
:102F7000FFF7C6FD0446FFF79BFDFFF751FE204615
:102F800070BD70B50446FFF725FEE0252846FFF723
:102F9000EDFDFFF771FE00B107E02046FFF7E6FD0B
:102FA000FFF76AFE00B100E000BFFFF739FE70BD19
:102FB00070472DE9F05F04460E46207800F00107C7
:102FC000207800F00208207800F00409207800F052
:102FD000080A207800F0100B002537B1012528469B
:102FE000FFF7CFFF012000F025FFB8F1000F06D05A
:102FF00002252846FFF7C5FF012000F01BFFB9F1AD
:10300000000F06D004252846FFF7BBFF012000F083
:1030100011FFBAF1000F06D008252846FFF7B1FFCF
:10302000012000F007FFBBF1000F06D01025284655
:10303000FFF7A7FF012000F0FDFEFFF78EFFA8427B
:1030400002D00020BDE8F09F35B164223146002057
:10305000FDF721F96420F5E70020F3E72DE9F05FA3
:1030600004460E46207800F00107207800F00208A0
:10307000207800F00409207800F0080A207800F099
:10308000100B002537B101252846FFF77AFF0120F4
:1030900000F0D0FEB8F1000F06D002252846FFF759
:1030A00070FF012000F0C6FEB9F1000F06D0042524
:1030B0002846FFF766FF012000F0BCFEBAF1000FC2
:1030C00006D008252846FFF75CFF012000F0B2FE7D
:1030D000BBF1000F06D010252846FFF752FF012054
:1030E00000F0A8FEFFF739FFA84202D00020BDE89B
:1030F000F09F2DB1642231460020FDF71AF9F6E762
:103100000020F4E71CB501210D2000F0E1F9542066
:10311000009000208DF8040001208DF806000320A7
:103120008DF8050000208DF8070069460F48FFF76D
:103130003CF94FF4A050009069460D48FFF735F96F
:103140004FF44070009001208DF807006946084850
:10315000FFF72BF969460748FFF727F94FF40040BE
:10316000009069460148FFF720F91CBD000C0240A1
:1031700000000240000802402DE9F04740212748A6
:10318000FFF77EF9054610212448FFF779F9064636
:1031900004212248FFF774F907464FF48051204874
:1031A000FFF76EF980464FF480611D48FFF768F91C
:1031B00081461C48007818B900250120194908707B
:1031C0001948007818B900260120174908701748D7
:1031D000007818B9002701201449087014480078B5
:1031E00020B94FF0000801201149087011480078FB
:1031F00020B94FF0000901200E49087045F0E000A9
:1032000040EA460040EA870040EAC80040EA091068
:10321000C043C4B22046BDE8F0870000000C024065
:1032200000000240A5000020A6000020A70000200A
:10323000A8000020A90000202DE9F0474FF40071FC
:103240007748FFF71DF904464FF480717448FFF783
:1032500017F905464FF400717248FFF711F9064659
:103260004FF480716F48FFF70BF907464FF40041A8
:103270006D48FFF705F9804644F0E00040EA45005C
:1032800040EA860040EAC70040EA0810C04300F068
:10329000FF094FF400716248FFF7F2F863490978BB
:1032A000884216D04FF400715D48FFF7E9F880B905
:1032B0001E2000F0BFFD4FF400715948FFF7E0F801
:1032C00038B90120FFF75DFE012000F0B3FDFFF7E4
:1032D00005FE4FF480715248FFF7D2F8544909783F
:1032E000884216D04FF480714D48FFF7C9F880B975
:1032F0001E2000F09FFD4FF480714948FFF7C0F891
:1033000038B90220FFF73DFE012000F093FDFFF7E2
:10331000E5FD4FF400714348FFF7B2F845490978DD
:10332000884216D04FF400713E48FFF7A9F880B9E3
:103330001E2000F07FFD4FF400713A48FFF7A0F81F
:1033400038B90420FFF71DFE012000F073FDFFF7E0
:10335000C5FD4FF480713348FFF792F8364909787C
:10336000884216D04FF480712E48FFF789F880B953
:103370001E2000F05FFD4FF480712A48FFF780F8AF
:1033800038B90820FFF7FDFD012000F053FDFFF7DD
:10339000A5FD4FF400412448FFF772F8274909784A
:1033A000884216D04FF400411F48FFF769F880B9F2
:1033B0001E2000F03FFD4FF400411B48FFF760F86E
:1033C00038B91020FFF7DDFD012000F033FDFFF7D5
:1033D00085FD4FF400711248FFF752F81349087049
:1033E0004FF480710E48FFF74BF8114908704FF405
:1033F00000710C48FFF744F80E4908704FF48071D3
:103400000848FFF73DF80C4908704FF400410648A2
:10341000FFF736F8094908704846BDE8F087000014
:103420000000024000080240000C0240A000002002
:10343000A1000020A2000020A3000020A400002082
:1034400070B504460D46052C00DC04B970BD601E45
:10345000C4B20121A140C8B2FFF793FD012000F0E2
:10346000E9FC2846FFF758FD00BFEFE72DE9F047DC
:10347000044604F00105C4F34006C4F38007C4F316
:10348000C008C4F3001929460120FFF7D9FF012025
:1034900000F0D0FC31460220FFF7D2FF012000F0FF
:1034A000C9FC39460320FFF7CBFF012000F0C2FC26
:1034B00041460420FFF7C4FF012000F0BBFC494651
:1034C0000520FFF7BDFF012000F0B4FCBDE8F08748
:1034D00029B1064A12680243044B1A6004E0034A09
:1034E00012688243014B1A60704700003038024076
:1034F00029B1064A12680243044B1A6004E0034AE9
:1035000012688243014B1A60704700004438024041
:10351000F0B5002100220024022500260223324FAC
:103520003F6807F00C0121B1042905D0082937D1E3
:1035300005E02E4F076036E02D4F076033E02A4F3D
:103540003F1F3F68C7F38056274F3F1F3F6807F074
:103550003F036EB1264FB7FBF3F7DFF88CC0ACF139
:10356000040CDCF800C0CCF3881C07FB0CF40CE066
:103570001E4FB7FBF3F7DFF870C0ACF1040CDCF8BA
:1035800000C0CCF3881C07FB0CF4174F3F1F3F68AB
:10359000C7F301477F1C7D00B4FBF5F7076002E02D
:1035A000124F076000BF00BF0F4F3F6807F0F001E8
:1035B0000909104F7A5C0768D74047600A4F3F6897
:1035C00007F4E051890A0B4F7A5C4768D74087605F
:1035D000054F3F6807F46041490B064F7A5C476826
:1035E000D740C760F0BD0000083802400024F40056
:1035F00000127A000701002001461C48814201D2D6
:10360000002070471A48814201D20820F9E7194882
:10361000814201D21020F4E71748814201D21820DC
:10362000EFE71648814201D22020EAE714488142A0
:1036300001D22820E5E71348814201D23020E0E79B
:103640001148814201D23820DBE71048814201D283
:103650004020D6E70E48814201D24820D1E70D48EC
:10366000814201D25020CCE75820CAE70040000830
:103670000080000800C000080000010800000208E7
:1036800000000408000006080000080800000A08FE
:1036900000000C0800000E0830B503460C46154625
:1036A000002206E0184600F007F844F822001B1D2F
:1036B000521CAA42F6D330BD01460868704700008C
:1036C0002DE9F04704460E4617464FF0090800253D
:1036D000A946B4F1006F02D304F0030008B1BDE8BD
:1036E000F087FEF73FFE0020FEF78AFD254604EB3B
:1036F00087091948854218D214E02846FFF7DCFFF5
:10370000401C70B1F120FEF775FD2846FFF774FFED
:1037100082460221FEF786FD8046B8F1090F01D0EE
:1037200002E02D1D4D45E8D300BFB8F1090F0CD1C3
:1037300008E020463168FEF7EDFD092800D003E0DF
:10374000241D361D4C45F4D300BF0120FEF758FD63
:10375000FEF7D6FD00BFC2E70000FF1F7047000064
:1037600030B500228B071C0F0F2303FA04F20B4B1A
:103770008C1053F824309343084C8D1044F82530B6
:1037800023468C1053F824308C07240F00FA04F4DD
:103790002343024C8D1044F8253030BD08380140D9
:1037A0000CB50020019000903448006840F480304F
:1037B0003249086000BF3148006800F400300090D2
:1037C0000198401C0190009818B90198B0F5A04FDD
:1037D000F1D12A48006800F4003010B101200090B7
:1037E00001E0002000900098012846D12348403095
:1037F000006840F08050214940310860204800684E
:1038000040F440401E4908601C48083000681B49CD
:10381000083108600846006840F400400860084627
:10382000006840F4A05008601648091F0860081F8F
:10383000006840F08070091F086000BF0F480068F2
:1038400000F000700028F9D040F205700E490860C1
:103850000A480830006820F0030008490831086071
:103860000846006840F00200086000BF03480830C6
:10387000006800F00C000828F8D10CBD00380240A8
:103880000070004008544007003C0240042808D162
:103890004FF0E021096941F004014FF0E02211618D
:1038A00007E04FF0E021096921F004014FF0E02228
:1038B000116170477047000010B51548006840F46A
:1038C0007000134908601348006840F00100114976
:1038D000086000200F49083108600E4800680E4952
:1038E00008400C4908600D48091D0860081F006861
:1038F00020F48020091F0860002006490C31086070
:10390000FFF74EFF4FF0006001498039086010BD9D
:1039100088ED00E000380240FFFFF6FE1030002482
:1039200010B50121054800F010F8012801D1044923
:1039300008700121014800F005F810BD00040040A6
:10394000AB000020CA430282704730B50246002017
:1039500000230024158A05EA0103958905EA01047C
:1039600013B10CB1012000E0002030BD70B5044659
:103970000D46FFF761FC00B21E490880FFF7FCFB13
:1039800000B21D490880012C10D11C48B0F900007C
:103990001849B1F90010884208D11948B0F900005F
:1039A0001549B1F90010884200D170BD1148B0F935
:1039B0000000124908801048B0F900001049088042
:1039C00002260C4800780F4908700B4800784870B0
:1039D0002A463146312000F017F90648B0F90000B8
:1039E000064908800448B0F900000549088000BF76
:1039F000DBE700009C0200209E020020A0020020C5
:103A0000A2020020B4460020002005E04FF6FF711E
:103A10000B4A22F81010401C1428F7DB002009493B
:103A2000087009490870094908700949086009497E
:103A300008700949088009490880094908807047C9
:103A400034570020AE000020AC000020AD00002064
:103A5000B0000020B4000020B6000020B800002014
:103A6000BA0000205E49098801F0200121B15C49BB
:103A7000091D0988C8B200E070475A4909780A2927
:103A80007BD2DFE801F00517232F353B4E52616DE5
:103A900055280ED10121544A1170544A1180002139
:103AA000534A118001214F4A117052490988524AE4
:103AB000118063E0AA2803D102214A4A117004E070
:103AC0000021494A1170474A117057E0BB2803D1C1
:103AD0000321444A117004E00021434A1170414A15
:103AE00011704BE004213F4A11704149088045E0C4
:103AF00005213C4A11703E4908803FE00621394AC1
:103B000011703B49098841EA0021394A118000219E
:103B1000364A11803649098811B90821314A117095
:103B20002CE007212F4A117000BF30490988491C39
:103B30002E4A1180114609882D4A1288914202DBD3
:103B40000821284A117019E00D2805D00021264AC5
:103B50001170244A117002E00921224A11700DE00F
:103B60000A2806D00021204A11701E4A117003E075
:103B700003E00A211B4A117000E000BF00BF1A4990
:103B8000097881B11B490A680968491C194B1960F9
:103B90001A4988541946096844F20802914202D32E
:103BA00000211A4611600F4909780A2915D11249D6
:103BB0000988134A134B1B7822F81310114909780E
:103BC000491C142291FBF2F302FB13110D4A1170F0
:103BD0000021054A1170034A117000BF4CE7000034
:103BE00000140140AE000020B4000020BA00002004
:103BF000B8000020B0000020B6000020AC06002075
:103C000034570020AC0000202DE9F04781460C46D7
:103C10001646274626B1A1B21048FEF7E4FD7F0004
:103C20000F4B3A460D494846FDF734FC804640218B
:103C30000C4800F019F800250CE00948415D0948DE
:103C400000F0C4F800BF4021064800F022F8012827
:103C5000F9D16D1C4545F0DBBDE8F087B446002086
:103C6000B44E00200014014001F40072B2F5007F50
:103C700000D100BFCA430280704721B1828942F45B
:103C80000052828104E082894DF6FF731A408281DE
:103C9000704702460020B1F5007F00D100BF1388B5
:103CA0000B400BB1012000E000207047F0B5034647
:103CB000002400260025002040F66A17B94200D1F2
:103CC00000BF1846C1F3421401F01F06012707FA8E
:103CD00006F5012C01D10C3004E0022C01D110308A
:103CE00000E014301AB107682F43076002E007684C
:103CF000AF430760F0BD00002DE9FF4705460E46C3
:103D00000024A14600BFA046B08900B100BF2C8AA4
:103D100024F44054F08804432C82AC8941F20C60B6
:103D20008443B08831890843718908430443AC81D6
:103D3000AC8A24F44074B0890443AC826846FFF72F
:103D4000E7FB2048854202D01F48854202D1DDF8BA
:103D50000C9001E0DDF80890A88900F4004040B123
:103D600009EBC90000EB091031684900B0FBF1F71D
:103D700007E009EBC90000EB091031688900B0FBCE
:103D8000F1F76420B7FBF0F004012009642101FB86
:103D90001078A88900F4004040B1322000EBC80040
:103DA000B0FBF1F000F00700044308E0322000EB24
:103DB00008106421B0FBF1F000F00F0004432C81E7
:103DC000BDE8FF870010014000140140C1F3080264
:103DD0008280704700BFFEE702E008C8121F08C1DA
:103DE000002AFAD170477047002001E001C1121F7C
:103DF000002AFBD17047000010B504466FF00400A4
:103E0000FFF744FDE11704EB5171C1F3C701074A05
:103E100011701046007800EB4001C1EBC0104FF666
:103E2000FF7101EAC0000249088010BD9C0000201B
:103E30009E00002070B504464FF4077094FBF0F02C
:103E4000C6B24FF4077094FBF0F100FB114085B24D
:103E500004B970BD05E04FF4077000F031F8701E32
:103E6000C6B2002EF7D115B1284600F029F800BFE0
:103E7000EFE700000146114A12784A434FF0E02371
:103E80005A6100229A611A46126942F001021A61CF
:103E900000BF4FF0E022106900F001021AB100F4F7
:103EA0008032002AF5D04FF0E022126922F00102A0
:103EB0004FF0E0231A6100229A6170479C000020B5
:103EC0000146114A12884A434FF0E0235A6100220A
:103ED0009A611A46126942F001021A6100BF4FF05E
:103EE000E022106900F001021AB100F48032002AC9
:103EF000F5D04FF0E022126922F001024FF0E023EA
:103F00001A6100229A6170479E00002010B5044695
:103F1000282221460148FFF7BFFB10BD0000010821
:103F200010B50446282221460148FFF7C9FB10BD01
:103F30000000010800B5A9B06846FFF7E7FF4FF0A1
:103F4000FF30CDF882006846FFF7EAFF0A20FFF74E
:103F500071FF29B000BD0000FEF740FFFEF7D0FB67
:103F60000024FDF7FDFCFDF7FBFC01212948FDF7CE
:103F70004FFC02212748FDF74BFC1F27A0460025D8
:103F80000CE0681CC2B239460420FDF729FE681C0B
:103F9000C2B241460520FDF723FE6D1C042DF0DB67
:103FA000FDF71AFB00260CE0642094FBF0F100FB07
:103FB000114008B9FEF792FE641C3220FFF75AFF49
:103FC000761CB6F57A7FEFDB0024FDF705FB1FE0DA
:103FD0003220FFF74FFF642094FBF0F100FB11400B
:103FE00008B9FEF77BFEFCF783FAFDF773FA0A487F
:103FF0000078012800D10BE0B4F57A7F06DB0121BF
:104000000846FFF7B3FCFDF7ABFC0024641C00BFBF
:10401000DEE70000FF7F2000840000200D480068DC
:1040200040F480200B4908600A481038006840F0CE
:104030001000084910390860032001218140064A18
:10404000430942F8231000BFBFF34F8FBFF36F8FB8
:104050007047000024ED00E000E200E010B588B0F9
:10406000044601210420FFF733FA01212020FFF745
:104070003FFA082206212548FEF7DFF9082207212A
:104080002248FEF7DAF9C020069002208DF81C00C5
:104090008DF81D0000208DF81E0001208DF81F00F6
:1040A00006A91A48FEF781F902940020ADF80C0029
:1040B000ADF80E00ADF81000ADF814000C20ADF80E
:1040C000120002A91248FFF717FE01211048FFF75E
:1040D000D4FD40210E48FFF7C7FD012240F22551D3
:1040E0000B48FFF7E3FD47208DF8040002208DF810
:1040F000050003208DF8060001208DF8070001A8B7
:10410000FEF7A6FEFFF780FC08B010BD00080240D5
:10411000001401403441020800000020AC020000FD
:1041200040020208A4420208AC020020046D000014
:10413000E83D020811130A08801732303233303953
:1041400031333038343232397A68616F796F6E6763
:1041500078104A6948654D736F3730303058326493
:104160003518810026394170702C526561645465A0
:104170006D70657261747572652C6E6577416E61E4
:104180006C6F67436F6D6D4D6F64657A0101011A45
:104190001506050806280B08060408060208060787
:1041A000080F1010060806030806010807030A078F
:1041B000050A07280A0A07040A07020A07070F1256
:1041C00008200D0C08040C08020C08070C10203CF9
:1041D0000501036B2C0203040419439209180832E9
:1041E0003032322D3031033D2030303A0311298BEB
:1041F0002DA10902080932022AC90C3129464BB502
:104200000A0C32044BA90B2432051AE10C29C432E2
:10421000061B190C0C3132071A5D0C292432155A71
:104220008D181993112AEB18312A21584A0D0C3296
:10423000225A050C32234B250E3032291A790C41B3
:1042400032302ADD0C191932314B510F0C32322A1F
:10425000690C3132331A810C299032342AF10C3135
:104260002A40544A100C32415AA50C32424B2D11AF
:104270000C32435AC50C2A48184A120C32505A6163
:104280000C32C14B09136C32E05A1D0C32E15A3525
:104290000C32E31A3D0C293032E44B19141801108A
:0442A0001AFF01817F
:040000050802018963
:00000001FF
